:0200000480007A
:10000000971F0000938F0F0137E0CDAB1300100056
:100010001360007F1370F0531340308013105000B2
:10002000135020401350400023A00F00971F0000E2
:10003000938F8FFE930010001301007F9301F05304
:1000400013023080930250001303200093034000FA
:100050001304800117E0CDAB3300100033602000A3
:100060003370300033404000331050003350604054
:10007000335070003300804023A00F00971F000012
:10008000938FCFF9930010001301200033A02000BC
:1000900023A00F0033B0200023A20F0013A02000E4
:1000A00023A40F0013B0200023A60F00971F000009
:1000B000938FCFF76F00400023A00F009700000040
:1000C0009380C0006780000023A20F0097100000FB
:1000D000938040F3971F0000938FCFF503A000009B
:1000E00023A00F000390000023A20F000380000054
:1000F00023A40F0003C0000023A60F001715000063
:10010000130545F1971500009385C5F3370610F0E8
:100110001306C6F26306B5028326C5002320D60067
:10012000832685002320D600832645002320D60081
:10013000832605002320D600130505016FF09FFDDF
:10014000370510F0130505F223200500000000001C
:0401500000000000AB
:101000004F4E5242000000000000000000000000AF
:10101000FFFFFFFFFFFFFFFFFFFFFFFFFFFFFFFFE0
:10102000FFFFFFFFFFFFFFFFFFFFFFFFFFFFFFFFD0
:10103000FFFFFFFFFFFFFFFFFFFFFFFFFFFFFFFFC0
:040000058000000077
:00000001FF
